:10000000830100308A000428203084004D301620FF
:1000100083010730D200FC30D1004D3084005130D4
:100020001A208301CA2C04068001840A0406031DD9
:1000300013280034F00026208000840A040870068B
:10004000031900341B2883120313D100D21B31285B
:10005000521B392852088A005108D10A0319D20AC2
:1000600082008313521883175108D10A84000008B4
:1000700008000A340D3424342534303431347834D3
:1000800020340034003482070A340D342A342034FA
:100090002834433429342034323430343034373443
:1000A0002C3420344F344C3449344D344534583496
:1000B00020344C347434643420342A3400348207BD
:1000C0000A340D342A342034503449344334203433
:1000D00049344F34203443344F344E345434523442
:1000E0004F344C3420342034203420342034203415
:1000F00020342A34003482070A340D342A342A3456
:100100002A342A342A342A342A342A342A342A34FF
:100110002A342A342A342A342A342A342A342A34EF
:100120002A342A342A342A342A342A3400348207DE
:0E0130000A340D342034453452345234003435
:10081C008301080083018C1E102C1A080800830128
:10082C00C200831203130C1E172C420899000800F7
:10083C00F0000030711870070310F00D0310F10C6C
:10084C00F10803190800202C8316031306118614D3
:10085C0090308312980024308316980081309900D0
:10086C00831208008301BF00C001432C40083F07DE
:10087C008400831300081524C00A40083F07840035
:10088C0083138008031908003C2CF401F5010310B4
:10089C00F30CF20C031C592C7008F40771080318A4
:1008AC00710AF5070310F00DF10D720873040319AA
:1008BC0000344D2C00308301061A0130BF000310A8
:1008CC00BF0D003086190130BF040310BF0D00307E
:1008DC0006180130BF040310BF0D0030051A01309B
:1008EC00BF043F080800FF308301BC070311031845
:1008FC00013E031DBD07FF3003110318013E031D0C
:10090C00BE07FF3003110318013E031DBF073F084C
:10091C003E043D043C0403190800792C8301C101F9
:10092C00A22C41083F07D1004008D20051080318FF
:10093C00D20A23201524C10A41083F07D1004008E0
:10094C00D20051080318D20A2320003803190800DA
:10095C00972C8301BC00BE01BD011024BD000D3AD3
:10096C00031DBE2C3E083C07840083138001080045
:10097C0008303E020318B32C3E083C078400831356
:10098C003D088000BE0AB32C80308316031381000F
:10099C008B01073083129F0083169F018612051668
:1009AC000614861506168511051185100510F030F4
:1009BC00831285052A247C30BF000030C0009424AB
:1009CC006030BF000030C00094244430BF000030C1
:1009DC00C00094247C30BF000030C00094244D3003
:1009EC0038242C30AF242C30FC24F52C8301BC0093
:1009FC00840083130008523A031D142D60248313C2
:100A0C00A2003930C0000030C1002208BD00BE0178
:100A1C003D30BF002430FF252430382C3C088400A6
:100A2C0083130008723A031D352D25301524061E3C
:100A3C00212D3130222D30301524861D272D3130BB
:100A4C00282D30301524061C2D2D31302E2D303014
:100A5C001524051E332D3130152C3030152C3C0847
:100A6C00840083130008573A031DC62D3C08023E30
:100A7C00840080080319912DFA2DF03085050508A6
:100A8C000800F030850505140800F0308505851444
:100A9C000800F0308505033085040800F03085052A
:100AAC0005150800F0308505053085040800F03088
:100ABC008505063085040800F0308505073085046F
:100ACC000800F030850585150800F03085050930E3
:100ADC0085040800F03085050A3085040800F030E4
:100AEC0085050B3085040800F03085050C30850435
:100AFC000800F03085050D3085040800F0308505C0
:100B0C000E3085040800F03085050F308504080090
:100B1C00F0308505FA2D3C0A840083130008303A26
:100B2C000319432D013A0319472D033A03194B2D91
:100B3C00013A03194F2D073A0319542D013A0319A1
:100B4C00582D033A03195D2D013A0319622D0F3A02
:100B5C000319672D013A03196B2D783A0319702D7F
:100B6C00033A0319752D013A03197A2D073A031923
:100B7C007F2D013A0319842D033A0319892D8E2DEB
:100B8C003C08840083130008773A031DFA2DA10159
:100B9C00A10AA301210883133C07840080080319D0
:100BAC00F72D053021020318EE2D0310A30D21089B
:100BBC003C0784000008313A031DE62D2314F52D63
:100BCC0021083C07840083130008303A0319F52DE3
:100BDC009830BF000030C0009424A301F72DA10A67
:100BEC00D02D2308850008009830BF000030C000CD
:040BFC00942C8301B1
:100C0000C800C6013F08C300AE2F4708253A031DA0
:100C1000A12FFF30C400C501C2016B2FC808031902
:100C2000152E48088400831380014608080002300E
:100C3000C30743028400831300089F2FC20A242E97
:100C40000830C407FE30C4070230C30743028400E3
:100C500083130008C900840A0008CA004218CA1F8A
:100C6000382EC909CA09C90A0319CA0AC503392E87
:100C7000C2010B30C4074408F200F3014A08F10036
:100C80004908F000C2277008C7004408F200F301C9
:100C90004908F0004A08F100C2277408C900750825
:100CA000CA00CB01CB0ACC014C084A02031D5A2EC4
:100CB0004B084902031C772E4408F200F3014B084D
:100CC000F0004C08F1004B247408CB007508CC00F0
:100CD000C503542EC60AC8080319752E4808840097
:100CE000831320308000C80A772E20300E24C503DD
:100CF0004508803A7F3E03186A2E421C8A2EC60A97
:100D0000C8080319882E4808840083132D30BB2E91
:100D10002D300E244408F200F3014B08F0004C087B
:100D2000F100C2277408CB007508CC004B040319EE
:100D3000C12E4C08F3004B08F2004A08F1004908A4
:100D4000F000C2277408F0007508F1004408F200B2
:100D5000F301C2277008C500803A763E031CB22E0C
:100D60000730C507C60AC8080319BE2E4808840004
:100D700083134508303E8000C80A8A2E4508303E5D
:100D8000892E0A304702031CC72E0730C707C60A40
:100D9000C8080319D12E4808840083134708303E41
:100DA000A92F4708303EAD2FC60AC8080319DF2E09
:100DB00048088400831320308000C80AE12E2030C8
:100DC0000E24C5034508803A7E3E0318D42E023017
:100DD000C3074302840083130008C700A12F023019
:100DE000C3074302840083130008CB00840A000871
:100DF000CC00C70147084B07D1004C08D20051086E
:100E00000318D20A232000380319082FC70AFA2E24
:100E10004408470203180E2F4708C4004408C51BA6
:100E2000392FFF3A4507031C392FC60AC808031992
:100E3000202F48088400831320308000C80A222F06
:100E400020300E24C5030E2F4C08D2004B0823205F
:100E5000C700CB0A0319CC0AC60AC8080319372FE2
:100E600048088400831347088000C80A392F4708C0
:100E70000E24C403440F242FAE2F4108D200400893
:100E800023202A3A031D4B2F0230C307430284005C
:100E900083130008672F4108D20040082320D03E6A
:100EA000C400C00A0319C10A4108D2004008232027
:100EB000C70030304702031C6B2F3A30470203183B
:100EC0006B2F0A30F10044081E244707D03EC400AF
:100ED000C00A0319C10A4108D2004008C00A031918
:100EE000C10A2320C700003A03190E2E2A3A03191B
:100EF000172E043A03193D2F763A0319202E3B3A58
:100F00000319E22E073A03191E2E0B3A0319222E5B
:100F10001C3A0319EF2E063A0319242E0D3A031931
:100F2000202E30304702031CA12F3A30470203180D
:100F3000A12F0A30F10045081E244707D03EC50006
:100F40006B2FC60AC8080319AC2F48088400831306
:100F500047088000C80AAE2F47080E244108D20077
:100F60004008C00A0319C10A2320C700C708031D8F
:100F7000052EC8080319C02F480884008313800178
:100F800046080800F601F401F50172087304031D18
:100F9000CC2FF001F10100341F30F6040310F60AE3
:100FA000F20DF30D031CCF2FF30CF20C730871023A
:100FB000031DDC2F72087002031CE42F7208F0027C
:100FC0007308031C730AF102F40DF50DF60BF61A03
:100FD000D42FF61FF02FF409F40A0319F503F509CD
:100FE0007408F2007508F300761F0034F009F00A67
:100FF0000319F103F10900340A340D343E3400348E
:02400E00223F4F
:00000001FF
